:020000040000FA
:1002000063EF01F09EA8FED70650AD6E1200ABA2C0
:1002100002D0AB98AB889EAAFED7AE50066E1200F5
:1002200089688A6A8B68F00E926E3F0E936E9F0EFD
:10023000946EC60EC16EC00EC26E400EAF6EFB0E47
:10024000AC14AC6E200EAC10AC6E100EAB10AB6EDE
:10025000800EAB10AB6E016A81B0FED7F00E036E5C
:10026000800E046E045000080EE20404046E010EB9
:100270000310036E020E0310036E040E0310036ED0
:100280000350896EEFD703688968026807EC01F0B4
:100290000650026E056A02A203D002A001D0052A10
:1002A000055202E1770E016E02B402D0F70E016E24
:1002B00002B602D07F0E016E0250896E0150066EAA
:0A02C00002EC01F0E2D710EF01F0AC
:020000040030CA
:0E000000FFFEF6FEFFFEFBFFF03FFF9FFFBF7F
:00000001FF
